:100000000C942A000C9445000C9445000C94450077
:100010000C9445000C9445000C9445000C9445004C
:100020000C9445000C9445000C9445000C9445003C
:100030000C9445000C9445000C9445000C9445002C
:100040000C9445000C9445000C9445000C9445001C
:100050000C94450011241FBECFE5D4E0DEBFCDBF18
:1000600010E0A0E6B0E0E2E3F2E002C005900D92FD
:10007000A036B107D9F710E0A0E6B0E001C01D92AC
:10008000A036B107E1F70C94E1000C940000CF9387
:10009000DF93CDB7DEB781E0809338001092350052
:1000A0001092320081E08093370010923400109259
:1000B0003100DF91CF910895CF93DF93CDB7DEB7B5
:1000C00026970FB6F894DEBF0FBECDBF69837A8343
:1000D0008B839C8389819A81AB81BC819C01AD011A
:1000E000689413F8220F331F441F551F1694D1F73D
:1000F00080E092E1AAE7B0E0BC01CD010E94F700E8
:10010000DA01C90101979E838D838D819E81892F9C
:100110009927809340008D818093290080912A0047
:10012000886180932A008091400086688093400017
:1001300026960FB6F894DEBF0FBECDBFDF91CF91EC
:100140000895CF93DF93CDB7DEB722970FB6F8941B
:10015000DEBF0FBECDBF80912B00882334F4809189
:100160002C0099279A83898302C01A821982898177
:100170009A8122960FB6F894DEBF0FBECDBFDF91F5
:10018000CF910895CF93DF93CDB7DEB721970FB608
:10019000F894DEBF0FBECDBF898380912B009927D5
:1001A00080729070009709F4F8CF898180932C00B9
:1001B00021960FB6F894DEBF0FBECDBFDF91CF9171
:1001C0000895CEE5D4E0DEBFCDBF0E94470060E8D1
:1001D00075E280E090E00E945C000E94A1008983AB
:1001E00089818823D1F389810E94C200F6CFA1E2E0
:1001F0001A2EAA1BBB1BFD010DC0AA1FBB1FEE1FA1
:10020000FF1FA217B307E407F50720F0A21BB30BEB
:10021000E40BF50B661F771F881F991F1A9469F767
:1002200060957095809590959B01AC01BD01CF01C3
:0202300008952F
:00000001FF
